:100000000200B9028003FFFFFFFFFF02800BFFFF2A
:10001000FFFFFF028013FFFFFFFFFF02801BFFFFB8
:10002000FFFFFF028023FFFFFFFFFF02802BFFFF88
:10003000FFFFFF028033FFFFFFFFFF02803BFFFF58
:100040003202147902149A021471021469021424FF
:1000500002158B0215B10214FA0214F70214EA0217
:1000600014C70214D60214AD0214AF0213FA02131D
:10007000CE0213A202138E02138602163702168BCB
:100080000216730216D50216E00216EB02151402D0
:10009000154B02152F02170302170702170B021741
:1000A0000F02171302171702171B02171F0213471D
:1000B0000217230217910216F975812F758922758F
:1000C0008DFDD28E759852C2B3C290121611D29085
:1000D000121611C290121611D290121611C290125D
:1000E0001611D29012161112134DF5F078A0F608E1
:1000F00076001214790D5342434D4F4E2076007412
:1001000031121471742E1214717433121471742E0E
:10011000121471743212147112147920496E6974B8
:1001200069616C697A65642E0D00E5F0B4FF1F12F9
:100130001479284E6F205852414D20776173206406
:100140006574656374656421290D0002017F1214D2
:10015000792844657465637465642000E912149A13
:100160001214796B206F66205852414D2061742023
:1001700000E5F012149A121479303068290D0075D8
:1001800090FF1214790D5342432052656164793E09
:100190002000121424FF9001C4E493600C6F6006E9
:1001A000A3A3A3A380F3A3E473121479496E766129
:1001B0006C696420636F6D6D616E643A2000121487
:1001C0001202017F3F0201FD41020C4949020B3638
:1001D00058020B3652020AD14C02096E4302083A09
:1001E0005602075D7702072A570206EA4D02065BB0
:1001F000450205B14B0204B951020AA70012147955
:100200000D53424320436F6D6D616E642053756DD5
:100210006D6172793A0D0D3F202D2054686973206D
:1002200068656C70206D656E750D41787878782002
:100230002D20537461727420617373656D626C69F3
:100240006E6720636F646520617420787878780D1C
:10025000435B7373206E6E2068682077206464208F
:100260006D6D2079795D202D2052656164204453A5
:100270003133303720525443205B6F7220736574E2
:100280005D0D455B746578745D202D205265616459
:10029000204154323530313041206D656D6F7279B7
:1002A000205B6F7220777269746520746578745D65
:1002B0000D4978785B2C79795D5B3D7A7A5B7A7A47
:1002C000207A7A207A7A5D5D202D20446973706CE3
:1002D0006179204952414D20787820746F207979D6
:1002E00020286F722073657420787820746F207ACC
:1002F0007A290D4B5B445D202D204B65797061643C
:100300002074657374205B4B443D44697361626C77
:1003100065206465626F756E63655D0D4C202D20F0
:100320004C6F6164204845582066696C6520696E91
:10033000746F205852414D0D4D5B307C317C325DE5
:100340005B495D202D20446973706C6179206D6F6D
:1003500064652C20303D4D656D6F7279206D617044
:100360007065642C20313D44697265637420382DBA
:100370006269742C20323D44697265637420342DA7
:100380006269742C20493D496E697469616C697AAF
:10039000650D5278787878202D20457865637574DE
:1003A0006520636F646520617420787878780D56D5
:1003B0005B465D202D20517569636B2074657374F5
:1003C000206F66205852414D203230303068202D49
:1003D000203346464668202856463D46756C6C20BC
:1003E00074657374290D575B546578745D202D20F6
:1003F0005772697465207465787420746F204C435B
:10040000440D775B61612062622063635D202D2073
:10041000577269746520636F6D6D616E64732061DE
:10042000612C62622C63632C206574632E20746FD0
:10043000204C43440D58787878785B2C7979797919
:100440005D5B3D7A7A5B7A7A207A7A207A7A5D5D92
:10045000202D20446973706C6179205852414D20E1
:100460007878787820746F207979797920286F727C
:1004700020736574207878787820746F207A7A29D0
:100480000D4E6F74653A20455343206174206265B8
:1004900067696E6E696E67206F66206C696E652095
:1004A00072657065617473206C61737420636F6D25
:1004B0006D616E640D0002017FC2981214790D4BBC
:1004C000657970616420746573743A2057696C6C47
:1004D000206563686F206B657970726573736573EF
:1004E00020746F2073657269616C20706F72740D77
:1004F000507265737320616E79206B6579206F6E21
:10050000205043206B6579626F61726420746F20A4
:100510007465726D696E6174650D007A0178B1E67B
:10052000601F7A001214794E4F54453A20444542D8
:100530004F554E43452044495341424C4544210DBB
:10054000007B0330980302017FEB9005AD93905040
:100550000EF582E0540F640F70061BBBFFE580E1CF
:10056000F9BA01107E177F00E0540F640F6970D153
:10057000DFF6DEF2C3E978001340030880FAC08298
:10058000C083EB23232890059D93121471D083D050
:1005900082BA0106E0540FB40FFA0205414142430A
:1005A0004433363923323538303134372A0E0D0B87
:1005B0000775F00078B1E6602AD2B2C0E0120627D3
:1005C000D0E0600605F008E680F112147957726FEA
:1005D000746520746F20454550524F4D0D00C2B2D6
:1005E00002017F12147952656164696E6720454586
:1005F00050524F4D3A2000120647600A12147105FE
:10060000F0E5F0B400F11214790D0002017FC294FC
:1006100074051214AF74FF1214AFD29422C29474F2
:10062000061214AFD29422C0E012060E540170F9E3
:1006300012061DC29474021214AFE5F01214AFD06A
:10064000E01214AFD29422C29474031214AFE5F0F6
:100650001214AF74FF1214AFD2942278B1E6C20024
:10066000C201B43106C201D2008007B43204D20103
:10067000D2001214794C4344206D6F646520736579
:100680007420746F20001206AD78B2E6B4491B12D4
:100690001479496E697469616C697A696E67204C76
:1006A00043440D0012151412152902017F20001376
:1006B0001214796D656D6F72792D6D61707065645E
:1006C0000D002212147964697265637420636F6E81
:1006D0006E65637420007438300102743412147132
:1006E0001214792D6269740D0022121479577269FF
:1006F00074696E67207465787420746F204C43446D
:1007000020001206AD78B1E6600612158B0880F75E
:100710001214794C434420577269746520636F6DDD
:10072000706C6574650D0002017F1214795772694F
:1007300074696E6720636F6D6D616E647320746F92
:10074000204C434420001206AD78B17A007B00793A
:10075000021213A240BAEB1215B10880EEC2987FC4
:100760001078B1E6700302076B7F0090800030982C
:100770000302081FEFF0A3E583B400F2908000307D
:10078000980302081FE0B5072AA3E583B400F0DF51
:10079000DA1214795852414D2074657374656420DF
:1007A0006F6B2038303030682D46464646680D0065
:1007B00002017FC0E0AA83AB821214795852414DE6
:1007C000204572726F725B00EA1213FA121471E81C
:1007D000121471EB1213FA121471E812147112143C
:1007E000795D3D00D0E01213FA121471E812147111
:1007F000121479202873686F756C642068617665BF
:10080000206265656E2000EF1213FA121471E8126F
:100810001471121479290D008A838B82020789C210
:10082000981214795852414D207465737420616296
:100830006F727465640D0002017F1214EA1214C70E
:1008400074D0C31214F7400E7400C31214F778B1B9
:10085000E660250209271214794E6F207265706CCC
:10086000792066726F6D204453313330372049430D
:100870000D0002017F0208751214C774D1C312144F
:10088000F740F2121479536563733A2000C31214CF
:10089000FA547F12149A1214790D4D696E733A202E
:1008A00000C31214FA547F12149A1214790D486F6F
:1008B00075723A2000C31214FA543F12149A12149B
:1008C000790D576461793A2000C31214FA12149A10
:1008D0001214790D4461793A202000C31214FA549D
:1008E0003F12149A1214790D4D6F6E74683A2000FD
:1008F000C31214FA541F12149A1214790D59656117
:10090000723A2000D31214FA12149A1214D6020169
:100910007F12147949324320436F6D6D2046617513
:100920006C740D0002017F12147953657474696E42
:1009300067205254430D007F077A007B0079021232
:1009400013A2400DEBBF0702547F1214F740C2DF21
:10095000E81214D6121479445331333037205254EC
:100960004320776173207365740D0002017F1209C3
:100970007402017F7D007C0012147953656E64203F
:10098000496E74656C204845582066696C6520691D
:100990006E207465787420666F726D6174206E6F5E
:1009A000772C204354524C2D5820746F2061626F75
:1009B00072740D00121469B41869121479496E74B6
:1009C000656C204845582066696C652075706C6FB1
:1009D0006164207761732061626F7274656420774F
:1009E000697468204354524C2D580D00D3221214C0
:1009F00079496E74656C204845582066696C65209D
:100A0000636F6E7461696E656420696E76616C698E
:100A10006420646174612C2061626F727465640D7E
:100A200000D322B43A8E12138E40C3FF2DFDEC3456
:100A300000FC12138E40B7F58312138E40B0F5827E
:100A400012138E40A9FEBE000912138E40A0F0A31F
:100A5000DFF7121469B40D028003B40AF5BE014435
:100A6000121479496E74656C204845582066696C8B
:100A7000652075706C6F616420636F6D706C657458
:100A8000652E0D00ECFEEDFF7C007D001216371286
:100A90001479206279746573206C6F616465642ECB
:100AA0000D00C3220209B4120974402212147945C0
:100AB0007865637574696E6720636F64652061741F
:100AC0002038303030680D00128000020B16020111
:100AD0007F121479457865637574696E6720636F5A
:100AE0006465206174200078B179021213A2EA12C1
:100AF00013FA121471E8121471EB1213FA12147132
:100B0000E81214711214790D00900B16C082C08384
:100B10008A838B82E4731214790D436F64652065B8
:100B20007865637574696F6E20636F6D706C657442
:100B3000650D0002017FD2F0BF4902C2F078B1E436
:100B4000FAFBFCFDFEFF79021213A2B42C08790413
:100B50001213A2020BD3B43D02805220F00B1214E8
:100B6000794952414D5B0080141214795852414D1D
:100B70005B00EA1213FA121471E8121471EB1213EB
:100B8000FA121471E81214711214795D3D0020F00C
:100B900005EBF8E680058A838B82E01213FA1214C3
:100BA00071E81214711214790D0002017F8A838B8F
:100BB000827C007D0079041213A2C0E020F007E5DA
:100BC00082F9EDF78002EDF0A3D0E0B400E38000FD
:100BD00002017F8A838B827E10BE103FAA83AB8284
:100BE00020F00C1214790D4952414D5B0080151212
:100BF00014790D5852414D5B00EA1213FA12147128
:100C0000E8121471EB1213FA121471E81214711233
:100C100014795D3D008A838B827E0020F005A882D6
:100C2000E68001E01213FA121471E81214717420B4
:100C3000121471E583B5040DE582B50508740D1233
:100C4000147102017FA30E809078B17904E4FCFD59
:100C50001213A2400778A0ECF608EDF678A0E61291
:100C6000149A08E612149A1214793A200078B07691
:100C700000121424700302017F9010847A00E49320
:100C80007016121479496E76616C6964206F706316
:100C90006F64650D00020C5C78B0E6B4000274204D
:100CA000121386F9C3E894B093697009E9B420027D
:100CB000800D0880E5A3A3A3A3A3A3A30A80BF0A72
:100CC0008A7F740693F57D757B00757E00E8FAEAED
:100CD000F8B60003020D9808E8FA900FEAEAF8E681
:100CE0007003020D98B423057FF00A800EB42F051F
:100CF0007FC00A8006E493702A7FE07C007D00EAD2
:100D0000F879041213A2400418020D541214794900
:100D10006E76616C6964206F706572616E640D003F
:100D2000020C5CE6B4000474208005B42C0274202C
:100D3000121386F9C3E89A93697009E9B420028016
:100D40000F0880B1A3A3A3A3A3A3A3A3A3020CDDB5
:100D5000740893FFE8FAE57EB40319121479546F0E
:100D60006F206D616E79206F706572616E64730DB6
:100D700000020C5CC0E0EF54F0B45006EF540F14C6
:100D8000F57BD0E075F003A424A2F9EFF709ECF7A6
:100D900009EDF7057E020CCFE57EB57D02802012BD
:100DA000147957726F6E67206E756D626572206F71
:100DB00066206F706572616E64730D00020C5CE5F5
:100DC0007FB42E0F78A0868308868278A4E6F0A3ED
:100DD000020F6DB42F0A78A38683088682020F6DF6
:100DE000757C009011CEE4937003020E88FBC082E4
:100DF000C083120FD4FCD083D082C0E07805790084
:100E0000A3BC00028011E493F654F0B450027901BF
:100E1000081C80EC020E77D0E0FCEBB57FF6BC003E
:100E200015E57B257CF57C78A2EDF678A5EEF678C5
:100E3000A8EFF6020EAAE9C0E078A27905ECFAE67E
:100E400054F0F5F0E7B4B00474E0801BB4B1028054
:100E5000F7B4B20280F2B4B30280EDB4D00474F0FF
:100E60008005B4D10280F7B5F00A09080808DACF86
:100E7000D0E080ADD0E0F9B90005057C020DE6E5D3
:100E80007C2408F57C020DE6121479496E76616CBB
:100E9000696420696E737472756374696F6E207310
:100EA000796E7461780D00020C5CE57C120FD478C9
:100EB000A08683088682E57CF0A378A2797EE7FF8E
:100EC0007003020F6DE6B4A1005003020F62B4B0CC
:100ED0003B08E6FA08E6FBE5822401E5833400548A
:100EE000F8F5F0EA54F8B5F020EBF0EA5407030304
:100EF00003F5F0C3E5829401F582E5839400F58360
:100F0000E045F0F0A3A3020F65020FA8B4B22F08CA
:100F100008E5822401FBE5833400FAC3E69BFB1855
:100F2000E69AFA600EB4FF13EBB48000400DF0A314
:100F3000020F65EBB48000500280F3020F77B4B16A
:100F40000C08E6F0A308E6F008A3020F65B4D1028E
:100F500080EFB4D0030880EDB4B30280F8B4C002CF
:100F600080F3080808DF03020F6D020EC578A0A603
:100F70008308A682020C5C12147952656C61746954
:100F800076652061646472657373206F7574206F79
:100F9000662072616E676520282B3132372F2D3124
:100FA0003238290D00020C5C1214794162736F6CA7
:100FB0007574652061646472657373206F757473F2
:100FC000696465206F6620326B20626C6F636B0D05
:100FD00000020C5C1490108475F007A42582F58241
:100FE000E58335F0F58374069322432020202020EA
:100FF000202010412020202020202020405230207E
:10100000202020203040523120202020204052300B
:10101000202020202020515231202020202020522A
:101020005232202020202020535233202020202004
:1010300020545234202020202020555235202020BA
:1010400020202056523620202020202057523720A2
:1010500020202020205840412B44505452206040F2
:10106000412B50432020207041422020202020206E
:10107000804450545220202020904044505452200C
:101080002020A0004E4F5020202000414A4D5020EB
:1010900020014C4A4D502020015252202020200196
:1010A000494E43202020014A424320202002414350
:1010B000414C4C20014C43414C4C200152524320A6
:1010C000202001444543202020014A4220202020A6
:1010D0000252455420202000524C20202020014163
:1010E0004444202020024A4E4220202002524554EF
:1010F00049202000524C43202020014144444320F9
:1011000020024A4320202020014F524C2020200260
:101110004A4E4320202001414E4C202020024A5AB2
:10112000202020200158524C202020024A4E5A20D4
:101130002020014A4D50202020014D4F56202020D4
:1011400002534A4D502020014D4F56432020024467
:10115000495620202001535542422020024D554C33
:10116000202020013F3F3F2020200043504C2020E2
:101170002001434A4E45202003505553482020016A
:10118000434C522020200153574150202001584306
:101190004820202002504F50202020015345544227
:1011A00020200144412020202001444A4E5A202082
:1011B00002584348442020024D4F565820200244F4
:1011C0004220202020014F52472020200100010210
:1011D000B003B10420052005B305300540055006D5
:1011E000B3B207B008B109200A200AB30A300A4096
:1011F0000A500BB3B202B00C0D200E20D00E20B35B
:101200000E20300E20400E20500FB3B207B0101148
:10121000201220D01220B312203012204012205071
:1012200013B202B014B32014B3D01420D01420B3DE
:1012300014203014204014205015B207B016B320EB
:1012400016B3D01620D01620B31620301620401624
:10125000205017B202B018B32018B3D01820D018FD
:1012600020B318203018204018205019B207B014AD
:1012700010B31A601B20D01BB3D01B30D01B40D042
:101280001B50D01CB202B01610B31D20701E801B64
:10129000B3B31BB3301BB3401BB3501B90D107B08B
:1012A0001BB3101D20601F20D01F20B31F20301F34
:1012B00020401F20501410C002B01B10B305902016
:1012C00080211B30B31B40B31B50B31610C007B0B6
:1012D00022B322102320D0B22320B3B22330D0B2C5
:1012E0002340D0B22350D0B224B302B025B325108E
:1012F00026202720B327203027204027205028B33E
:1013000007B029B329102A202BB3B22C20302C206F
:10131000402B50B22D20A002B02D20302D20402592
:10132000201B20B31B20301B20401B20502DA02051
:1013300007B02D30202D402022201BB3201B302051
:101340001B40201B502000740D75F002229080007D
:10135000E0C0E0121378D0E0F040057480793222CA
:1013600090E000E0C0E0121378D0E0F0400574E0B7
:1013700079082274FF7900227800E8F0E0687004B0
:10138000D8F8C322D322B46100400254DF221214E1
:10139000691213CE400BC4F91214691213CE400126
:1013A0004922D2D5E61213CE401FC2D5C0E0E7C411
:1013B00054F0F709E754F0C41947F709E7540FC48C
:1013C000F7D0E047F7190880DBE608A2D522B43051
:1013D000004025B43A005004540FC322B4410040E9
:1013E00017B447005004C3943722B461004009B4D5
:1013F0006700500454DF80EED322F8540F24F650D7
:10140000022407243AC8C4540F24F65002240724A7
:101410003A2278B0E6600712147108B800F6740D2D
:101420001214712278B0C2983098FDE599B408156D
:10143000B8B00280F1121471742012147174081281
:1014400014711880E1B40D09760012147178B0E6B9
:1014500022B40A0280D0B41B04740D80EDB8FF02E0
:1014600080C4121471F60880BD3098FDE599C298C9
:1014700022C299F5993099FD22D083D082C0E0C074
:10148000D0C299E493A36009F5993099FDC299807F
:10149000F2D0D0D0E0C082C08322C000C0E01213DE
:1014A000FA121471E8121471D0E0D0002274FFC057
:1014B00007D296C2977F08A2E79295D297A296C2CA
:1014C0009733DFF3D00722D291D29212162BC2911A
:1014D000121625C29222C291121625D29212162BF2
:1014E000A092D29112162BA091227A09C3C2921215
:1014F00014D65002DAF622D3800274FFC0027A09B1
:1015000033929112162BD292121625A291C292DA20
:10151000EFD00222743830010274281215B1740E13
:101520001215B174061215B12274011215B12220E0
:10153000000C904003E0C0E012154BD0E022D2B581
:10154000121559C0E012154BD0E02220000990403E
:1015500002E020E7FC8018C2B5D2B43001051215B4
:10156000708009D2B37590FFE590C2B320E7E822FE
:101570004390F0D2B3E590C2B354F0C0E0D2B3E5EB
:1015800090C2B354F0C4FFD0E04F22C0E0C083C08B
:1015900082200006904001F0800DC2B4D2B58024B4
:1015A000F590D2B300C2B312154BD082D083D0E0F5
:1015B00022C0E0C083C082200006904000F080116D
:1015C000C2B4C2B5200114F590D2B300000000C22D
:1015D000B312154BD082D083D0E022C0E0440F4339
:1015E00090F05290D2B300000000C2B3D0E0C444E7
:1015F0000F4390F05290D2B300000000C2B380D1EC
:10160000C006C0077E027FDFDFFEDEFAD007D0060D
:1016100022C006C0077E027F32121600DFFBDEF713
:10162000D007D00622000000000022C0077F0C1265
:101630001625DFFBD00722C083C082790078041210
:101640001673600812168B09C0E080F1B9000574AA
:101650000009C0E0D0E02430121471E914600D7567
:10166000F00384E5F07005742C121471D9E6D08271
:10167000D08322C0F088F0C0F08AF0E47A044608F3
:10168000DAFCAAF0D0F0A8F0D0F022C0F088F0C0C8
:10169000F08AF0C0F08BF0C0F0E675F00A84F6E551
:1016A000F0C4F5F0087A03E6C4540F45F075F00A6B
:1016B00084C4FBE5F0C4D675F00A844BF6E5F0C4AB
:1016C000F5F008DAE2C4D0F0ABF0D0F0AAF0D0F038
:1016D000A8F0D0F022C3EF33FFEE33FEED33FD224E
:1016E000C0E0EF2BFBEE3AFAD0E0221216E0C0E0A9
:1016F000ED39F9EC38F8D0E02275F00A8443F03087
:1017000044302290500E2290500D2290500B229087
:1017100050072290400022904001229040022290E7
:10172000400322C0F0EFC0E0EEC0E0EBC0E0E9C053
:10173000E0C083C0827B03EB9005AD93905000F531
:1017400082E0540F640F70071BBBFFEBE4802BF9A2
:101750007E177F00E0540F640F6970D9DFF6DEF268
:10176000C3E978001340030880FA79ABA78379AC0A
:10177000A782EB23232890059D93F5F0D082D08398
:10178000D0E0F9D0E0EBD0E0EED0E0EFE5F0D0F043
:1017900022C0E0E8C0E0C083C08278AB868378AC2A
:1017A0008682E0540FB40FFAD082D083D0E0F8D014
:1017B000E022FFFFFFFFFFFFFFFFFFFFFFFFFFFF35
:00000001FF
